:020000020000FC
:020000005AC0E4
:020016003EC0EA
:10001A0000C04F935F930F935FB7409167004530DD
:10002A000CF403C0442740936700403041F493988E
:10003A0094989598929A00916600B5D06BD0413009
:10004A0041F4929894989598939A00916500ABD050
:10005A0061D0423041F4929893989598949A00917D
:10006A006400A1D057D0433041F492989398949861
:10007A00959A0091630097D04DD0439540936700BD
:10008A005FBF0F915F914F9118950F930FB7B29B76
:10009A0005C0B39B05C0B49B05C005C0019603C04B
:1000AA000A9601C0CF960FBF0F9118950FED0DBF9D
:1000BA000EE701BB01EC07BB0CE108BB00E20BBF7A
:1000CA000CE100BD02E000BF05E003BF09E106BF85
:1000DA0001E009BF11241092670080E090E026D069
:1000EA00789449D070FD969A70FF9698FACFEE24CC
:1000FA00FF1841E1001F111F4A9509F40895EE1CEB
:10010A00FF1CE21AF30A20F4E20EF31E8894F2CFDF
:10011A000894F0CF0F930FB800E40EB90BE10DB9B4
:10012A00769BFDCFC09AC0980F910895F89400E08D
:10013A000CBD0CE30ABD05E408BD03E00EBDB99A87
:10014A0008B706FFFCCFB99808B705FFFDCF0DD059
:10015A0000E00CBD04E30ABD08B706FFFDCF002787
:10016A000EBD0FEF08BF78940895B19B7160089592
:10017A00F894789408955F9354E0A3E6B0E08093EE
:10018A0061009093620000916100109162002AE080
:10019A0030E0ADDFED9200936100109362005A9552
:1001AA0091F75F9108950F931F93EAEEF1E01127FB
:1001BA00E00FF11F04901F910F91089503EB0A9528
:1001CA00F1F708950F931F930FEF1FEF1A95000091
:1001DA0000000000D9F70A95C1F71F910F91089501
:0C01EA00C0F9A4B0999282F880909C00AB
:00000001FF
